:020000040000FA
:1000000041EF02F0F76A140FF66E000EF7220900B6
:10001000F5501200C0F9A4B0999282F880908883BC
:10002000C6A1868EFF0E926E3F0E936EA00E946E4A
:10003000000E956E968096829684C150C00B07097B
:10004000C16EC050C00B0209C06EC09EC280000EBF
:10005000016EC250C30B0110C26EC2828B940C0E93
:10006000BD6EB76A000E0409CA6EFF0ECB6E7F0E1E
:10007000BE6EA1EF02F07F0E08010F6F116B106BC7
:10008000156B146B070E176FFF0E166F000183EFD1
:1000900000F07F0E08011A6F1B6B1C91000185EFA9
:1000A00000F00801876B875121081AE31ED8360E2D
:1000B0008825E96E080E8921EA6EEF6A16D8010ECE
:1000C0008825016E000E8921036E0150360FE96EFE
:1000D000080E0320EA6EEF6A0400872B53EF00F04E
:1000E000010E586F000187EF00F0D8908735896BBB
:1000F000886F12007F0E08017E6F000189EF00F00B
:100100008A8E3BEF00F049EF00F051EF00F07AEFFC
:1001100000F08B80000E956ED50E8C6EA3EF02F072
:100120000850F00B08018E6F09382ED88B6F0A50DB
:10013000F00B8E6F0B3828D88C6F0CC08DF88D5358
:1001400002E1800E8D6F11518B15126F10C813F8DC
:10015000125113031FD88C031DD88D1504E0FF0E18
:100160000F6FB4EF00F00F6B8A5306E01051D8B454
:1001700011071007BFEF00F0102BD8B4112B0FC8D8
:1001800001F00001E6EF02F0006E0F0E00160050C5
:100190008E251200F3500F6F0F5112000850F00B14
:1001A00008018E6F09382FD88B6F0A50F00B8E6FB5
:1001B0000B3829D88C6F0CC08DF88D5302E1800E5E
:1001C0008D6F11518B15126F10518C15136F1251C9
:1001D0001303F3500F6F0F518D1504E0FF0E0F6FD7
:1001E000F3EF00F00F6B8A5306E01051D8B41107FB
:1001F0001007FEEF00F0102BD8B4112B0FC801F040
:100200000001F4EF02F0006E0F0E001600508E2574
:100210001200036A080183D8EF3C13EF01F07F0E50
:10022000016E8CEF01F02651D8B42707260726531C
:1002300019E1275317E1036A72D8D890276BEF3082
:10024000266F0D50FF0A006ED8900032005026270E
:10025000000E2723265305E1275303E1276B010EE8
:10026000266F251F2951D8B42A072907295320E1D1
:100270002A531EE1036A53D8D8902A6BEF30296FB6
:100280000C50FF0A2927000E2A230B5209E02A539B
:1002900003E129512E5D04E22E51295F000E2A5BF5
:1002A000295305E12A5303E12A6B010E296F281F08
:1002B0002C51D8B42D072C072C530FE12D530DE1F1
:1002C000D8902D6B0A302C6F200E2C27000E2D237A
:1002D0002B51040802E2040E2B5F2F51D8B43007D3
:1002E0002F072F530AE1305308E1306B0BC02FF872
:1002F0002E51010802E2010E2E5F1CA184EF01F0D5
:10030000FF0E2B6F2E6F1C91255128030FD81A5109
:100310002B030CD81AC801F00001FCEF02F01B51AE
:100320001D0FE96E080E0320EA6E1200F3508B6F6A
:10033000F4CF8CF88CC81AF81200083808018B6FBB
:100340008B33070E8B1709C08CF88C1F32518C5DD4
:1003500009E0036A8B511D0FE96E080E0320EA6E57
:100360008CC8EFFF8CC832F83107315302E0CBEF75
:1003700001F07F0E316F8A5308E01B071B510708FD
:1003800002E2070E1B6FCAEF01F01B2B1B5107087F
:10039000D8A01B6B1C8100011DEF03F00801906BBE
:1003A000095063D88B6F8B333F0E8B178D6B0AC050
:1003B0008CF85FD85ED85DD85CD8F00E8C170850EA
:1003C00054D88E6F8E333F0E8E170B308F6F8F3356
:1003D0008F331F0E8F178007805309E18BC880F879
:1003E000805304E1FF0E7F6FF7EF01F07F1F8D5107
:1003F000835D05E303E182518C5D01E23DD88251CA
:10040000D8B48307820782530BE1835309E134D8C0
:10041000825305E1835303E1836B010E826F811FD9
:10042000813D15EF02F08FC890F88507855310E1E4
:100430008EC885F88551905D04E29051855F23EF69
:1004400002F0010E856F855302E1010E856F841F56
:100450007F5304E17F0E7E6F30EF02F084C87EF898
:100460007EC801F000011AEF03F0FF0A006E0030B1
:1004700012008C378D3712008DC883F88CC882F833
:100480001200F86AD08E7E0E006E100E016E020E03
:10049000E96E000EEA6EEE6A002E4BEF02F0012EBE
:1004A0004BEF02F0EA6AE96A720EEDD8C150C00B58
:1004B0000F09C16E070EB46E7F0E056E0E6A7F0EB9
:1004C00008010F6F106B116B126B136B146B156BB4
:1004D000FF0E166F070E176F186B196B7F0E1A6FD2
:1004E0001B6B1C91256B010E266F276B286B010E71
:1004F000296F2A6BFF0E2B6F010E2C6F2D6BFF0ED9
:100500002E6F010E2F6F306B316B326B336B010E20
:10051000346F356B010E7C6F7D6B1C937F0E7E6F8D
:100520007F6B010E806F816B010E826F836B846B1A
:10053000010E856F010E866F700EA5D8000112EFB7
:1005400000F080EF00F0D1800801876B88910638B9
:10055000876F87338733030E8717889181B8888127
:100560008751020816E10838006E0032070E0016A7
:100570000050010F036AF2CF8BF8F29CF29E00014B
:1005800041DD08018BBDF28C8BBFF28E8C6ECBEF00
:1005900002F0D50E8C6E81BAD0EF02F01EEF03F0A0
:1005A0008751000108E0010A14E0030A20E0010A73
:1005B00032E01DEF03F00801860704E000011DEFA3
:1005C00003F00801075064D890EF00F06DD81DEFDC
:1005D00003F00801860704E000011DEF03F00801A5
:1005E000075056D8CEEF00F05FD81DEF03F0000E95
:1005F00008015DD809EF01F057D80801860704E02B
:1006000000011DEF03F00801075056D83F0E5AD8DD
:100610004ED89DEF01F00801860704E000011DEFB0
:1006200003F00801075048D886331F0E4BD83FD837
:10063000CEEF01F039D81DEF03F0080105C0BEFF71
:10064000C2B23FEF03F0C282036A0E50060FE96E9A
:10065000000E0320EA6EC2B22BEF03F0C4CFEFFF0F
:100660000E2A0E500708D8A00E6A0E34006E00360F
:10067000FC0E0016C250C30B0010C26EC2820400F2
:10068000A5EF02F00300D36E400E9B6ED350120014
:10069000FF0A006ED8900030866F862B000E88B15E
:1006A000010E8A6F0001120001C005F0120088B12E
:1006B000010E8A6F00011200FF0A006E0030866F83
:0C06C000863312008617862B000E1200F5
:020000040030CA
:0E0000000008180F008381000FC00FE00F40B2
:00000001FF
